:1023E60020000A3C2E2E2E3E004950436F6E6E652D
:1023F60063745245510A004950436F6E6E656374AB
:10240600000A49504E6F41434B210A003E432C5669
:102416002C43432CC0E4E0EFF2E5F020D1E8EDEAEE
:10242600EEEC49500A003E432C4D41432C253032F8
:1024360062583A25303262583A25303262583A2587
:10244600303262583A25303262583A253032625874
:102456002C4D414320E0E4F0E5F10A003E432C56C2
:1024660045522C20332E3220EEF220257320257380
:102476002CC2E5F0F1E8FF20495020ECEEE4F3EB46
:10248600FF0A004D61722031332032303132003183
:10249600363A34323A3137003E432C4C442C5052B3
:1024A6004F473A20202020202020202020202020B6
:1024B6002020202020202020202020202020202016
:1024C6002020202020202020202020202020202006
:1024D60020202020202020202020202020202020F6
:1024E60020202020202020202CC4E0F2E020EFF045
:1024F600EEF8E8E2EAE828F4E0E9EB290A003E2AE9
:102506002C312CCEF1EDEEE2EDFBE520EFE0F0E034
:10251600ECE5F2F0FB20F1E5F2E5E2EEE3EE20E891
:10252600EDF2E5F0F4E5E9F1E00A003E412C413038
:10253600312C2562752E2562752E2562752E256233
:10254600752C495020E0E4F0E5F120E0E4E0EFF2FC
:10255600E5F0E00A003E412C4130322C2562752E12
:102566002562752E2562752E2562752C495020E050
:10257600E4F0E5F120EEF1ED2E20F1E5F0E2E5F0F4
:10258600E00A003E412C4130332C2562752E25622F
:10259600752E2562752E2562752C495020E0E4F0D3
:1025A600E5F120F0E5E72E20F1E5F0E2E5F0E00ABE
:1025B600003E412C4130342C2562752E2562752E45
:1025C6002562752E2562752CCCE0F1EAE020F1E556
:1025D600F2E80A003E412C4130352C2562752E2545
:1025E60062752E2562752E2562752CD8EBFEE70ADC
:1025F600003E2A2C312CC4EEEF2E20EFE0F0E0EC6A
:10260600E5F2F0FB20F1E5F2E5E2EEE3EE20E8ED9F
:10261600F2E5F0F4E5E9F1E00A003E422C533031F0
:102626002C2562752CC6E4E0F2FC20E7E0EFF0EE24
:10263600F1E020F1EEE5E4E8EDE5EDE8FF20EEF26D
:1026460020F1E5F0E2E5F0E00A003E422C5330329C
:102656002C2562752CCEE1ECE5ED20F120F1E5F0BC
:10266600E2E5F0EEEC20E1E5E720EAE2E8F2E0ED73
:10267600F6E8E90A003E422C5330332C2562752CCD
:10268600CFE5F0E5E7E0EFF3F1EA20EFF0E820EF41
:10269600EEF2E5F0E520F1E2FFE7E820F120F1E5D2
:1026A600F0E2E5F0EEEC0A003E422C5330382C25E1
:1026B60062752CCCE5E4EBE5EDEDFBE92049502015
:1026C600EAE0EDE0EB28E7E0E4E5F0E6EAE020E426
:1026D600EE203520F1E5EA290A003E422C5330353A
:1026E6002C2562752CCAE0EDE0EB20F8E8F0EEEA66
:1026F600EEE2E5F8E0F2E5EBFCEDEEE3EE20EEE1EE
:10270600ECE5EDE00A003E532C5330362C253032F2
:10271600625825303262582530326258253032628E
:1027260058253032625825303262582C4D414320AC
:10273600E0E4F0E5F120F8E8F0EEEAEEE2E5F8E0B4
:10274600F2E5EBFCEDEEE3EE20EEE1ECE5EDE00A82
:10275600003E454E440A000A44756D7058202020FC
:1027660020203030203031203032203033203034B9
:102776002030352030362030372030382030392090
:102786003041203042203043203044203045203034
:1027960046000A3A003A20000A000A44756D704461
:1027A600202020202030302030312030322030339D
:1027B6002030342030352030362030372030382055
:1027C6003039203041203042203043203044203000
:1027D6004520304600457272206B657900526420B0
:1027E600656570726F6D0A005264204D454D0A0092
:1027F600526420436F64650A00577269746520430A
:102806006F64650A0044656275674950204F4E0A39
:102816000044656275674950204F46460A00446584
:1028260062756755736572204F6E0A00446562755E
:102836006755736572204F46460A004465627567A0
:102846004D7367204F6E0A0044656275674D736766
:10285600204F46460A00436F6E666967206C6F63B9
:102866006B210A00577220656570726F6D0A002031
:102876005361766520656570726F6D210A00457239
:1028860072204D414321004C6F61643E3E002A0098
:10289600CEF8E8E1EAE00A00202D20257528257506
:1028A600290A003C4130313D003C4130323D003C7C
:1028B6004130333D003C4130343D003C4130353DF4
:1028C600003C21003C5330313D003C5330323D004A
:1028D6003C5330333D003C5330353D003C5330389B
:0828E6003D003C5330363D007B
:064F9E00011300011100E7
:10527800C28E438910E4F58B758DB8D2ABD28E22DD
:03001B000246D5C5
:1046D500C0E0C083C082C0D0C28E758B00758DB816
:1046E500201A0675A61E75A6E10511D216E51360FA
:1046F5000205130516E516540F7051E512D3940102
:1047050040021512D222E516543F7012D21490665B
:104715008EE0600A04F0E0D394B44002D21A9066A9
:1047250087E0600204F0906104E0600214F0906696
:104735008FE0D394014003E014F03019020514E52D
:1047450015D394644004D21A80020515E510D3945C
:104755000140021510D28ED0D0D082D083D0E03265
:10115900C291C290D2B5C21F7D027C007F07125195
:10116900F68F26E526646060097D017F601251696A
:10117900D21FE4FDFC7F0B1251F68F26E52630E6DF
:10118900097D04E4FF12518DD21F7D017C007F0788
:101199001251F68F26E5267008FD7FFF125169D29C
:1011A9001F301F03126000C288C2A8C2AA75890035
:1011B900124B1B90633FE0B4FA06A3E064CE607B58
:1011C900E4F52674372526F582E43463F583E4F0E3
:1011D9000526E526B443EC90633F74FAF0A374CE78
:1011E900F0A374CCF0906345740AF0E4A3F0A3046F
:1011F900F0A3F090633B74FFF0A3F0A3F0E4A3F035
:101209009063567403F0E4F526E5262401FFE433E0
:10121900FE74372526F582E43463F583E0FD125127
:10122900B10526E526C3944340DFE4F5A775A61E5C
:1012390075A6E1907FF0F0A3F080FE90634A7403F5
:10124900F0A374CCF0E4906349F090668CF0A3F0BD
:101259001240D1C2B5123BCFC21A124E08D21FC2D8
:1012690021C2209065777408F09062B57424F0E487
:10127900A3F090633FE09062B7F0906340E0906222
:10128900B8F0906341E09062B9F0906342E09062F7
:10129900BAF0906343E09062BBF0906344E09062DF
:1012A900BCF0751201E4906578F0C21BC21CC21D26
:1012B900C21E201F18AF26FE7D031241B7E4FF129C
:1012C90044DA7E237FE6E4FBFDFC123CDA90668E6D
:1012D900E060037401F0E4906104F0F51490657620
:1012E900F0F51512527875A70775A61E75A6E1D2F5
:1012F900AFE4F515906104E070031217E190668F71
:10130900E06401701D9080007410F09080A874FF53
:10131900F0A3F0A3F0A3F0E490668FF0D21FC220EF
:10132900C221908008E0F52630E405D21B7410F044
:10133900E52630E508D21D9080087420F0E52630B6
:10134900E608D21C9080087440F0E514C394034069
:1013590019908002E4F0908001F0908000F0E5148B
:1013690094064006E4F514124E089080A0E070033C
:10137900124C819080B8E07003124B999080D0E0B4
:101389007003124DAC908000E07013301B10123EB8
:10139900E5906332EFF0D394004003120036908059
:1013A90002E07006908000E06005D2190212FAC2CC
:1013B90019E4F514906104E060030212FA201F1287
:1013C900906579E0600C7E237FE8123FE9E490653F
:1013D90079F0301D12123817906332EFF0D3940070
:1013E9004005E0FF1252D4201C0302157E12350D70
:1013F900906332EFF070030212FA906376E054BF03
:10140900247F70030214D91470030214B1240260FA
:1014190003021520201F077E237FEF123FE92023B7
:101429000302157E90634EE07006906352E0606798
:10143900906683E0FF90634EE0B50724906684E0F0
:10144900FE90634FE0B50618906685E0FE90635004
:10145900E0B5060C906686E0FE906351E06E603759
:10146900906352E06F600302157E906684E0FF90FE
:101479006353E06F600302157E906685E0FF906319
:1014890054E06F600302157E906686E0FF90635515
:10149900E06F600302157EC2179065787401F0123F
:1014A900001E75120102157E90668EE060037401BC
:1014B900F090667BE0FF906378E06F600302157E31
:1014C90090667BE004F0E4F512906576F002157EF3
:1014D90030170302157E906345E070030212FA90FB
:1014E90062B4E06008906356741EF08006906356FB
:1014F9007403F01252C3D217E4F512906576F09096
:10150900668704F0E490667AF0A3F0201F677E23D3
:101519007FFD123FE9805E90668EE060037401F002
:10152900301752906376E020E74B906378E0FF90A4
:10153900667AE0FE6F600D906682E07007EE146FC8
:101549007033801390667AE004F0906332E0FFD341
:10155900940440031252D59060007482F0A3740180
:10156900F0906378E0906002F07E607F007D031266
:1015790049060212FA2017030216A1E512706E122B
:101589004765EF60237E647F76906477E02404FDED
:10159900124906906682E07009906356E0F51202DE
:1015A90012FAE4F5120212FA906687E0D3943C40ED
:1015B9003C906682E070369062B4E0703090668745
:1015C90004F0124373E4906476F0A37412F0906609
:1015D9007BE0906478F0A374FDF090610563A2014B
:1015E90090647A63A2017F121230D180981252D18D
:1015F9008F26E526B401159060007483F0E4A3F00A
:101609007E607F007D021249060212FAE526D39414
:1016190001401C9060007483F0A37401F0E5262456
:10162900FEA3F07E607F007D031249060212FAE5EF
:1016390012640160030212FA906576E004F0201F3B
:10164900077E247F07123FE9906576E0FFD3940176
:10165900400B906356E0941E5003E004F0EFC394EE
:1016690005400DC217E4906578F012001E0212FAC7
:101679007C667D8390634AE0FAA3E0FB7F02124A0D
:10168900977E647F76906477E02404FD1249069082
:101699006356E0F5120212FAE512640160030212C0
:1016A900FA906578E014604624FE604214700302E3
:1016B9001794240460030212FAE4F514202313900A
:1016C90065787404F0906576E05401F075120102B2
:1016D90012FA9080027410F0E4906578F0906576C3
:1016E90004F075121290668374FFF00212FA906684
:1016F90083E0700302177E9064767480F0906478BA
:101709007401F0E4A3F0A304F0A37430F0A3747B94
:10171900F0E4F526747D2526F582E43464F58374B6
:101729007DF0747E2526F582E43464F583E4F0E5E2
:10173900262407906477F07C667D8390634AE0FAFB
:10174900A3E0FB7F02124A977E647F76E52624098F
:10175900FD124906906682E0601B1252C3D217E45B
:10176900F512906576F090668704F0E490667AF059
:10177900A3F00212FA302307E4906578F08006900E
:1017890065787404F07512120212FA9080027410CE
:10179900F0751203906576E06401FFF09065787446
:1017A90001F0EF7019906352E06013FCA3E0FDA310
:1017B900E0FEA3E0FF90668312107C0212FA9063A8
:1017C9004EE0FCA3E0FDA3E0FEA3E0FF90668312D8
:0717D900107C0212FA80FEF1
:0117E00022E6
:10003600906377E0B444047F0180027F009063768A
:10004600E0B447047E0180027E00EE5F604A906362
:100056003FE0906378F0906340E0906379F09063BE
:1000660041E090637AF0906342E090637BF09063A6
:1000760043E090637CF0906344E090637DF090638E
:10008600777452F09062AE63A2019080A863A201D9
:100096007F061230D1020917906332E0C3940850EC
:1000A6000302092090633FE0FF906378E06F6003EE
:1000B600020920906340E0FF906379E06F600302DD
:1000C6000920906341E0FF90637AE06F60030209C4
:1000D60020906342E0FF90637BE06F60030209209B
:1000E600906343E0FF90637CE06F60030209209019
:1000F6006344E0FF90637DE06F6003020920906334
:1001060077E06444701A9080A8E0B4FF139062AE62
:1001160063A2019080A863A2017F061230D18010ED
:100126009062B2E09080ACF09062B3E09080ADF067
:1001360090668EE060037401F090668F7464F090B0
:1001460063777452F0906376E0646D60030202BADE
:100156007BFF7A2479121229507BFF7A24792C901E
:10016600633FE0F530A3E0F531A3E0F532A3E0F517
:1001760033A3E0F534A3E0F5351229507530FF7549
:1001860031247532897533FF7534247535957BFFB7
:100196007A2479621229507BFF7A24799E1229509B
:1001A6007BFF7A2579041229507BFF7A25793190D5
:1001B6006345E0F530A3E0F531A3E0F532A3E0F5C1
:1001C600331229507BFF7A25795B90634EE0F53038
:1001D600A3E0F531A3E0F532A3E0F5331229507B15
:1001E600FF7A257989906352E0F530A3E0F531A3D3
:1001F600E0F532A3E0F5331229507BFF7A2579B773
:1002060090633BE0F530A3E0F531A3E0F532A3E0DF
:10021600F5331229507BFF7A2579DA906337E0F5BA
:1002260030A3E0F531A3E0F532A3E0F5331229500F
:100236007BFF7A2579F71229507BFF7A267920A24F
:1002460023E433F5301229507BFF7A2679509066E5
:1002560082E0F5301229507BFF7A26797B90668EF4
:10026600E0F5301229507BFF7A2679AE9062B4E031
:10027600F5301229507BFF7A2679E0A215E433F592
:10028600301229507BFF7A27790C90667CE0F53096
:10029600A3E0F531A3E0F532A3E0F533A3E0F534AE
:1002A600A3E0F535122950123AAF7BFF7A2779572A
:1002B60012295022906376E0644C70737E277F5D2E
:1002C600FBFDFC123CDA90637EE0F527A3E0F528FF
:1002D600E4F52AE527906380F0A3E528F07E277FE2
:1002E600987C637D807B02123CDAE4F529852882BE
:1002F600852783E0FF74802529F582E43463F5833E
:10030600EFF00528E528700205270529E529B41030
:10031600DC7E277F9B7C637D807B10123CDA052A7E
:10032600E52AC3941040AC7E277F9E123FE92290B7
:100336006376E0646C7060F52B7E277FA0FBFDFC86
:10034600123CDAE4F52AE4906380F0A3E52BF07E14
:10035600277F987C637D807B02123CDAE4F529A82E
:100366002BE6FF74802529F582E43463F583EFF0EC
:10037600052B0529E529B410E67E277F9B7C637D46
:10038600807B10123CDA052AE52AC3940840B77E22
:10039600277F9E123FE922906376E0644B7061F5F9
:1003A6002974682529F582E43463F583E0603274A4
:1003B600682529F582E43463F583E0F460237468E4
:1003C6002529F582E43463F583E0FF747E2529F55B
:1003D60082E43463F583E0B507100529E529B408FE
:1003E600C09061047432F00209179063767421F0AC
:1003F600301F030209177E277FDB123FE902091728
:10040600906376E0B4521A201F077E277FE3123FDF
:10041600E99063767472F07E637F767D0812487F7A
:1004260022906376E064497045201F077E277FEEA1
:10043600123FE990637EE0F527A3E0F528E4F5296D
:10044600852882852783E0FF74802529F582E43498
:1004560063F583EFF00528E528700205270529E5F1
:1004660029B480DC7E637F767D8A12487F22906382
:1004760076E064437046201F077E277FF6123FE929
:1004860090637EE0F527A3E0F528E4F52985288228
:10049600852783E493FF74802529F582E43463F588
:1004A60083EFF00528E528700205270529E529B41C
:1004B60080DB7E637F767D8A12487F22906376E0BA
:1004C600645A7053201F077E277FFF123FE990630F
:1004D6007EE0F527A3E0F5287C637D807B80AF284E
:1004E600AE2712504BE4F529852882852783E493AD
:1004F600FF74802529F582E43463F583EFF005283F
:10050600E528700205270529E529B480DB7E637F8F
:10051600767D8A12487F22906376E0644460030207
:1005260005AE90637EE0FF64447003020917EFB4E2
:10053600310CC21F7E287F0B123FE9020917906318
:100546007EE0B4300CD21F7E287F17123FE90209E5
:100556001790637EE0B4320CD2207E287F24123FAF
:10056600E902091790637EE0B4330CC2207E287F2F
:1005760032123FE902091790637EE0B4340CD221AF
:100586007E287F41123FE902091790637EE0B43569
:100596000CC2217E287F4E123FE902091790637E26
:1005A600E0FF120032020917906104E07013201F69
:1005B600077E287F5C123FE99063767421F002097A
:1005C600179061047432F0906376E0FFB45104C270
:1005D600AF80FEEF64577045201F077E287F6A12A2
:1005E6003FE990637FE0906332F0E4F5299063324F
:1005F600E0FFE529C39F400302091774802529F50A
:1006060082E43463F583E0FF90637EE0252924AD20
:10061600F582E43461F583EFF0052980D0906376A6
:10062600E0645360030206D1201F077E287F7512FF
:100636003FE990633FE0FF9061B6E06F703C9063E6
:1006460040E0FF9061B7E06F7030906341E0FF904B
:1006560061B8E0B50724906342E0FF9061B9E0B568
:100666000718906343E0FF9061BAE0B5070C90630A
:1006760044E0FF9061BBE06F60169063767421F0F2
:10068600301F030209177E287F84123FE9020917EB
:10069600E4F529E4F515AF29FE74AD2529F582E4C4
:1006A6003461F583E0FD1251B10529E529C394FEB5
:1006B60040E1C2AFE4907FF0F0A3F0907FFD74AA12
:1006C600F0A374FFF0A37455F080FE906376E064A7
:1006D6004F705A90637EE0F527A3E0F528E528459C
:1006E60027700A201F077E287F8D123FE9201F07EB
:1006F6007E287F94123FE9E4F52974802529F58246
:10070600E43463F583E0852882852783F00528E5B0
:1007160028700205270529E529B480DE90668DE05C
:100726002480F090668CE03400F00209179063761E
:10073600E06445707490637EE0FEA3E0FF907FF076
:10074600EEF0A3EFF0D39400EE94044038907FF0DF
:10075600E0FEA3E0FF90668CE0FCA3E0FD9FEC9E2C
:100766004023E42FFFEE3401FED3ED9FEC9E50159F
:10077600C2AF907FFD74AAF0A374FFF0A37455F086
:10078600E4F5A780FE7E287F96123FE97BFF7A2854
:10079600799E907FF0E0F530A3E0F53190668CE02D
:1007A600F532A3E0F533122950906376E064656074
:1007B6000302092090637EE0FFA3E0907FF0CFF074
:1007C600A3EFF0E4F527F528D3907FF1E095289084
:1007D6007FF0E095274020E4F5152528FFE527342E
:1007E60001FE852882852783E0FD1251B10528E5A3
:1007F600287002052780D17E287FA912498DEF4EE9
:100806006020120003906345EFF0120003906346E8
:10081600EFF0120003906347EFF012000390634875
:10082600EFF07E287FAF12498DEF4E602012000355
:1008360090634EEFF012000390634FEFF012000347
:10084600906350EFF0120003906351EFF07E287F23
:10085600B512498DEF4E6020120003906352EFF0FF
:10086600120003906353EFF0120003906354EFF00D
:10087600120003906355EFF07E287FBB12498DEF7F
:100886004E602012000390633BEFF012000390636A
:100896003CEFF012000390633DEFF012000390630B
:1008A6003EEFF07E287FC112498DEF4E6020120088
:1008B60003906337EFF0120003906338EFF01200F5
:1008C60003906339EFF012000390633AEFF0E4F51A
:1008D60029E4F515E5292401FFE433FE74372529BB
:1008E600F582E43463F583E0FD1251B10529E5296B
:1008F600C3944340DCC2AFE4907FF0F0A3F0907F56
:10090600FD74AAF0A374FFF0A37455F0E4F5A78074
:0A091600FE7E637F767D0812487FA5
:0109200022B4
:104FDE00AE07EEC39430400BEED394395005EE2459
:104FEE00D0FF22EEC39461400BEED394665005EED3
:104FFE0024A9FF22EEC39441400BEED394465005F4
:08500E00EE24C9FF22AF0622C7
:10524C009062ADE004F070069062ACE004F0906205
:0A525C00ACE0FEA3E0FF12521322A3
:1000030012524C124FDEEFC454F0FEC00612524C93
:08001300124FDED0E02FFF22A6
:104D4F00E4906875F012524C906876EFF0C394308F
:104D5F004018E0FFD394395011906875E02405F5A1
:104D6F0082E43461F583EFF08011906875E02405DB
:104D7F00F582E43461F583E4F0800C906875E0040B
:104D8F00F0E0D3940840BE752B00752C00752D00F4
:0C4D9F00E4F52E7B017A6179051231DF0A
:014DAB0022E5
:04498D008E2C8F2DB0
:104991009062ACE4F0A374FFF012524CEF606EF43D
:1049A100606B852D82852C83E493B507EC752E0110
:1049B100E52D252EF582E4352CF583E493602590D1
:1049C10062ADE0252EFF9062ACE03400FE1252137E
:1049D100E52D252EF582E4352CF583E493B5070406
:1049E100052E80CCE52D252EF582E4352CF583E4CA
:1049F1009370A6E52E24FFFFE434FFFE9062ADE044
:104A01002FF09062ACE03EF07E007F0122E4FEFFD9
:014A11002282
:1040D1007E287FC712498DEF4E70037F01227E2813
:1040E1007FCA12498DEF4E600C12524CEF24D0243E
:1040F100FF92238002D2237E287FD012498DEF4E7A
:10410100600C12524CEF24D0906682F08005E4904E
:104111006682F07E287FD612498DEF4E600C1252D6
:104121004CEF24D090668EF08005E490668EF07E90
:10413100287FDC12498DEF4E600C12524CEF24D0D7
:1041410024FF92158002C2157E287FE212498DEF6D
:104151004E600C12524CEF24D09062B4F08005E412
:104161009062B4F090633F63A20190667C63A20108
:104171007F061230D130153B7E287FE812498DEF42
:104181004E603012000390667CEFF01200039066DF
:104191007DEFF012000390667EEFF012000390664F
:1041A1007FEFF0120003906680EFF012000390663B
:0641B10081EFF07F002207
:104F1000906577E0C3947C40027F0A906577E0FE5D
:104F200004F074B52EF582E43462F583EFF0BF0A25
:104F300027906577E0FF04F074B52FF582E43462C2
:104F4000F583E4F0906577E0FF124A12906577747C
:094F500008F09062B6E004F022C2
:104CEF0075B180E4F5B3F5B2854FBCE5505403FFC1
:104CFF0033333354F8FFE55054E04FFFE551C413FD
:104D0F0054074FF5BDE55133333354F8FFE552C423
:104D1F001354074FF5BEE55233333354F8F5BF85BF
:104D2F0054A38555A38556A38557A38558A38559A5
:104D3F00A3855AA3855BA3E553540F2450F5B322E3
:104E620043AB01C2E8C2EAE4FFEFC454F0F5B1E497
:104E7200F5B3F5B2F5BCF5BDF5BEF5BFF5C4F5C5A4
:104E8200F5C6F5C7F5A3F5A3F5A3F5A3F5A3F5A319
:104E9200F5A3F5A30FBF0ED190689DE0FF25E0F5C5
:104EA200B475B50C75B66C75A11275AB0275C13EC1
:064EB20075C3FF75C20389
:014EB80022D7
:02504B008B2CAC
:10504D00A2AF9224C2AF85A22D53A2FE8E838F8272
:10505D0005A28C838D8274091231CDE52C53A2FEED
:10506D0043A2201231CF53A2DF852DA2A22492AFED
:01507D00FF33
:01507E00220F
:1051F600A2AF9224C2AF8C838D82EF1231CD43A22F
:0C520600201231CF53A2DFA22492AFFF90
:015212002279
:025169008F278E
:10516B00A2AF9224C2AFE4F5838D8274061231CDC7
:10517B00E52743A2201231CF53A2DFA22492AF7FA7
:01518B000122
:01518C002200
:02518D008F276A
:10518F00A2AF9224C2AFE4F5838D82740A1231CD9F
:10519F00E52743A2201231CF53A2DFA22492AF7F83
:0151AF0001FE
:0151B00022DC
:101E3E003E2A2C312CC4E0F2F7E8EA20F2EEF7ED60
:101E4E00EEE3EE20E2F0E5ECE5EDE82E20CFE0F05B
:101E5E00E0ECE5F2F0FB20EFEEF0F2E0204750531D
:101E6E002E200A003E4C2C4930312C256C752CD17D
:101E7E00EAEEF0EEF1F2FC20EEE1ECE5EDE02C35D1
:101E8E00302C3130302C3330302C3630302C313247
:101E9E0030302C323430302C343830302C3936301F
:101EAE00302C31393230302C33383430302C353709
:101EBE003630302C3131353230300A003E532C471B
:101ECE005030302C2562752CCFE5F0E8EEE420EA98
:101EDE00EEF0F0E5EAF6E8E820E2F0E5ECE5EDE814
:101EEE002C20F1E5EA2E2028302E2E323535290A07
:101EFE00003E532C475030372C2562642CCFEEFF1A
:101F0E00F1EDEEE520F1ECE5F9E5EDE8E5204341F4
:101F1E004E2C20F7E0F12E200A003E532C47503075
:101F2E00382C2562642CCFEEFFF1EDEEE520F1ECBE
:101F3E00E5F9E5EDE8E52045544845524E45542C6B
:101F4E0020F7E0F12E200A003E2A2C312CCFE0F0B3
:101F5E00E0ECE5F2F0FB20EFEEF0F2E02043414E34
:101F6E002E200A003E4C2C6B30312C25732C43EA6C
:101F7E00EEF0EEF1F2FC20EDE020F8E8EDE5204386
:101F8E00414E2C30202D20353030EAE1283530EC12
:101F9E00292C31202D203530EAE128353030EC293E
:101FAE000A0030202D20353030EAE1283530EC297A
:101FBE000031202D203530EAE128353030EC290073
:101FCE003E2A2C312CC4E0F2F7E8EA20F2E5ECEFE1
:101FDE00E5F0E0F2F3F0FB2E20CDE0F1F2F0EEE9C9
:101FEE00EAE820EFEEE4EAEBFEF7E5EDE8FF2E205F
:101FFE000A003E422C475030352C2562752CCFE519
:10200E00F0E5E4E0E2E0F2FC20F2E5ECEFE5F0E0F2
:10201E00F2F3F0F30A003E422C475030392C256281
:10202E00752CC4E0F2F7E8EA20F2E5ECEFE5F0E01B
:10203E00F2F3F0FB20E820E2EBE0E6EDEEF1F2E861
:10204E002053485431780A003E4C2C475030312CE6
:10205E00256C752CCAEEEBE8F7E5F1F2E2EE20E422
:10206E00E0F2F7E8EAEEE220F2E5ECEFE5F0E0F27E
:10207E00F3F0FB2C312C322C332C342C352C362C0B
:10208E00372C380A003E4C2C475030322C256C75BC
:10209E002CC1FBF2FC20E1EBEEEAEEEC20D2C8D232
:1020AE002C302C312C322C332C342C352C362C3726
:1020BE000A003E4C2C475030332C256C752CC3F047
:1020CE00F3EFEFE020EFE0F0E0ECE5F2F0EEE22CE3
:1020DE00302C312C322C332C342C352C362C370A18
:1020EE00003E532C475030342C2562752CCFE5F032
:1020FE00E8EEE420EEE1EDEEE2EBE5EDE8FF2C207C
:10210E00F1E5EA2E28302E2E32353029200A003EF7
:10211E00532C475030362C2562752CCCE0F1F8F25A
:10212E00E0E1EDFBE920EAEEF4F4E8F6E8E5EDF2A5
:10213E00200A003C21003C4930313D003C6B3031DF
:10214E003D003C475030303D003C475030313D0063
:10215E003C475030323D003C475030333D003C4709
:10216E005030343D003C475030353D003C475030F8
:10217E00393D003C475030363D003C475030373DEE
:10218E00003C475030383D000AC2F0E5ECFF20ED30
:10219E00E020F1E5F0E2E5F0200A000AD2E5ECEFEE
:1021AE00E5F0E0F2F3F0E020EDE020F1E5F0E2E51D
:1021BE00F0200A000AC2F0E5ECFF20554E49583ACD
:1021CE00200A000A537461727420534854207465B7
:1021DE006D706574617475726520636F6E7665726D
:1021EE0073696F6E000A5348542074656D70657480
:1021FE00617475726520636F6E76657273696F6E4A
:10220E00206661696C75726521000A53746172747F
:10221E00205348542068756D696469747920636F22
:10222E006E76657273696F6E000A53485420687536
:10223E006D696469747920636F6E76657273696F08
:10224E006E206661696C75726521002025322E3212
:10225E00662064656772656573000A53485420747E
:10226E00656D706574617475726520636F6E7665E9
:10227E007273696F6E20636F6D706C657465202D5F
:10228E0020000A5348542068756D6964697479207A
:10229E00636F6E76657273696F6E20636F6D706CAF
:1022AE00657465202D20000ACEF2EFF0E0E2EAE040
:1022BE0020E22043414E20EEF2ECE5EDE5EDE0218B
:1022CE00000AD6E8EAEB20E8E7ECE5F0E5EDE8FFFA
:1022DE0020F2E5ECEFE5F0E0F2F3F0FB000AC8EDDA
:1022EE00E8F6E8E0EBE8E7E8F0F3FE20F2E5F0ECE4
:1022FE00EEECE5F2F0200A00202D2020EDE5F22094
:10230E00EEF2E2E5F2E000202D20204F4B21000AF4
:10231E00D1F2E0F0F220EFF0E5EEE1F0E0E7EEE2F0
:10232E00E0EDE8FF20E4E0F2F7E8EAE020000ACE74
:10233E00F2EFF0E0E2EAE020E22043414E20E7E057
:10234E00E2E5F0F8E5EDE021000ACFEEEBF3F7E57C
:10235E00ED20EFE0EAE5F2205542583A200A000A55
:10236E00CEF2EFF0E0E2EAE020F2E5ECEFE5F0E0AD
:10237E00F2F3F0FB20E22043414E200A000AD2E5A0
:10238E00ECEFE5F0E0F2F3F0E020F1EBE8F8EAEE46
:10239E00EC20F0E5E7EAEE20E8E7ECE5EDE8EBE02F
:1023AE00F1FC202D20EEF2E1F0E0F1FBE2E0FE2068
:1023BE00000AD2E5ECEFE5F0E0F2F3F0E020F120D8
:1023CE00E4E0F2F7E8EAE0200020ECE8EDF3F1209B
:0823DE000020EFEBFEF12000EE
:104FA4000163780167005066C10000000000000042
:104FB40000000000000000000048684400000000F9
:104FC4000000000052669000000000000000000095
:094FD400000000000000000000D4
:0100320022AB
:10437300E4FF0F2405F582E43461F583E564F00F6F
:1043830074052401F582E43461F583E4F07C667DF1
:1043930095FEED1DAA0470011CF5828A83E0FBAA39
:1043A300070F74052AF582E43461F583EBF00EBE42
:1043B30004E07C667D99E4FEED1DAA0470011CF502
:1043C300828A83E0FBAA070F74052AF582E434612D
:1043D300F583EBF00EBE04E07C667D9DE4FEED1DEF
:1043E300AA0470011CF5828A83E0FBAA070F7405F7
:1043F3002AF582E43461F583EBF00EBE04E07C66BB
:104403007DA1E4FEED1DAA0470011CF5828A83E000
:10441300FBAA070F74052AF582E43461F583EBF0F8
:044423000EBE04E0E5
:014427002272
:024428008F32D1
:10442A00908001E030E5099065797402F07F0022FE
:10443A003006037F0022D206906899E0FCA3E0FDD3
:10444A00A3E0FEA3E0F5368E358D348C3390667C7E
:10445A0063A201E535540744C8F58385368263A211
:10446A00017F06123159E5362406F536E43535F56D
:10447A0035E43534F534E43533F53390657A63A29F
:10448A0001E535540744C8F58385368263A201AF36
:10449A0032123159E4FCFDFEE5362532F536EE35A9
:1044AA0035F535ED3534F534EC3533F53390804C4C
:1044BA00E533F0A3E534F0A3E535F0A3E536F0AF34
:0F44CA0036AE35AD34AC3390689912107CAF32FA
:0144D90022C0
:0C0026003006089080017420F0C2062211
:0300230002398817
:10398800C0E0C083C082C0D075D018209803023A26
:103998008BC298300003023AA6301103023AA630CF
:1039A8000359301031E599640D601E74E02565F502
:1039B80082E43467F583E599F00565E565D394629B
:1039C8004014C291C203023AA6D200D205C203C271
:1039D80010C291023AA630022274E02565F582E40D
:1039E8003467F583E599F00565E565C3955F500390
:1039F800023AA6D211C203C202C291300E6474E028
:103A08002565F582E43467F583E599F00565E56594
:103A1800C394075003023AA6C20E9067E1E06462BD
:103A2800701AA3E0B40115A3E0B42110D203D202A6
:103A3800A3E02565547FF55F055F80629067E2E04B
:103A48006447701AA3E0B45015A3E0B45210A3E081
:103A5800B44D0BA3E0B44306D203D2108040C29108
:103A6800803CE599B42407D291756502D20EE59998
:103A780064B5702AD2919067E0E599F0756501D236
:103A88000E801BC299300116AF62056274762FF55D
:103A980082E43464F583E0F599D56602C201D0D09A
:073AA800D082D083D0E03290
:0300330002501662
:10501600C0E0C0F0C083C082C0D075D00830DC12BA
:10502600124CEF120026D207C2DCC2AEC20AC20D73
:105036008008C2D8C2D9C2DAC2DBD0D0D082D0832F
:05504600D0F0D0E032C3
:1051D500AB07E4FD7F9012511340107FAC12514193
:1051E5007F091251411252987F00221252987F0175
:0151F5002297
:10523000AB07E4FD7F90125113400B7FEE125141FA
:0C5240001252987F00221252987F012227
:103AAF007BFF7A1E793E122950906873E0FEA3E0E7
:103ABF00FFC3E49FFFE49EFEAB07FA3395E0F9F8EE
:103ACF007F007E8C7D0A7C00120FCB8F338E328D60
:103ADF00318C307BFF7A1E79721229507BFF7A1E50
:103AEF0079CA9066A2E0F5301229507BFF7A1E79D1
:103AFF00FF855D301229507BFF7A1F792885613051
:103B0F001229507BFF7A1F795612295090689DE039
:103B1F0070147530FF75311F7532B07BFF7A1F79C6
:103B2F007212295080127530FF75311F7532BF7BAD
:103B3F00FF7A1F79721229507BFF7A1F79CE1229D3
:103B4F00507BFF7A207900A204E433F5301229501C
:103B5F007BFF7A207924A209E433F5301229507BB8
:103B6F00FF7A2079569066D4E0FFE48F33F532F573
:103B7F0031F5301229507BFF7A207993906864E0F9
:103B8F00FFE48F33F532F531F5301229507BFF7A90
:103B9F002079C09066D1E0FFE48F33F532F531F52F
:103BAF00301229507BFF7A2079EF90684CE0F53086
:103BBF001229507BFF7A21791D85693012295022F5
:103383007E217F4112498DEF4E70037F01227E2102
:103393007F4412498DEF4E6023124D4FA804A905B7
:1033A300AA06AB077F007E8C7D0A7C00120FCB122E
:1033B300105D906873EEF0A3EFF0800A9068737469
:1033C300FFF0A374B8F0E490689DF07E217F4A1269
:1033D300498DEF4E601B12524C8F27E527B43106FF
:1033E30090689D740AF0E527B4320690689D746472
:1033F300F07E217F5012498DEF4E600A124D4F909F
:1034030066A2EFF080069066A27405F07E217F57D6
:1034130012498DEF4E6017124D4F8F27E527C39446
:1034230009500280027F089066D4EFF08006906610
:10343300D47402F07E217F5E12498DEF4E600F122D
:103443004D4FEF5407FFE4906864EFF080069068F7
:10345300647407F07E217F6512498DEF4E600F1271
:103463004D4FEF5407FFE49066D1EFF0800690666E
:10347300D17407F07E217F6C12498DEF4E600A12E2
:103483004D4F90684CEFF0800690684C741EF07EB0
:10349300217F7312498DEF4E600C12524CEF24D0F2
:1034A30024FF92048002C2047E217F7A12498DEFA9
:1034B3004E600C12524CEF24D024FF92098002C2BA
:1034C300097E217F8112498DEF4E6007124D4F8F88
:1034D300698003756901E56970037569017E217F60
:1034E3008812498DEF4E6007124D4F8F5D8003E4C4
:1034F300F55D7E217F8F12498DEF4E6007124D4F90
:093503008F618003E4F5617F0093
:01350C00229C
:103BCF00C296D20BE4F55CC290C20FC291C20A90AA
:103BDF00687374FFF0A374F4F0E490689DF075605F
:103BEF00FFF568756409C207123383C2089066A295
:103BFF00E09067DBF090684CE0FCE4120BC9E4FB4B
:103C0F00FA79C87842120A19E4FBFA7980784212DD
:103C1F000B22120BFD9066D9EEF0A3EFF09066D455
:103C2F00E075F005A490685DF0C206124E62C2AD59
:103C3F00E4F5C9D2CDD2CCC2C9C2CAF5CDF5CC906C
:103C4F006873E0F5CBA3E0F5CA85CBCD85CACCE48C
:103C5F00F598D29EC2ACC298C29975B81075B710BC
:103C6F00D2CAD29CD2ACD296C2A94389014388044E
:103C7F00F5D975DE3175D84075B740D2AF9066D59E
:103C8F00F09066D4E0FFA3E0C39F5035E0FF246BB4
:103C9F00F582E43468F5837401F01251D59066D53E
:103CAF00E0FE24ACF582E43466F583EFF074A32EC6
:103CBF00F582E43466F583EFF09066D5E004F0808A
:0B3CCF00C0E49066ABF09066D2F022DB
:0752C300D2CAD29CD2AC223A
:0152D40022B7
:104F590090657A7448F0A37461F0906864E0906594
:104F69007CF09066D1E025E025E0FF9066D5E0FE73
:104F79002F248090657DF0A37402F0EE25E024C112
:104F8900F582E43466F583E0FEA3E090657FF0EEF8
:054F9900A3F07F0722D8
:103DE100AF61EF3395E0FE7C0E7D10120E78EE335D
:103DF10095E0FDFC906865E0F8A3E0F9A3E0FAA383
:103E0100E02FF531EA3EF530E93DF52FE83CF52E9E
:103E1100302408752C65752D7A8006752C68752DF2
:103E21004D052DE52DAE2C7002052C14F5828E83E7
:103E31007401F0052DE52DAE2C7002052C14F582D0
:103E41008E837418F0052DE52DAE2C7002052C140F
:103E5100F5828E837480F0052DE52DAE2C70020560
:103E61002C14F5828E837401F0052DE52DAE2C7096
:103E710002052C14F5828E837406F0052DE52DAE16
:103E81002C7002052C14F5828E83E531F0052DE5A9
:103E91002DAE2C7002052C14F5828E83E530F005D1
:103EA1002DE52DAE2C7002052C14F5828E83E52FA5
:103EB100F0052DE52DAE2C7002052C14F5828E83B4
:103EC100E52EF0052DE52DAE2C7002052C14F582A2
:103ED1008E83E4F0852D82852C83F03024057F0BC1
:033EE10012442860
:013EE40022BB
:10476500300743C207C224123DE1E4906476F07538
:10477500270BA3740BF090667BE0906478F0A3742C
:1047850009F090684D63A20190647A63A201AF2796
:104795001230D1C21330210B7E217F96E4FBFDFC44
:1047A500123CDA7F012230134220AE3FE49064765A
:1047B500F0124F598F27906477EFF090667BE09069
:1047C5006478F0A37409F090657A63A20190647A25
:1047D50063A201AF271230D1C21330210B7E217F96
:0D47E500A9E4FBFDFC123CDA7F01227F00FD
:0147F20022A4
:0152D50022B6
:05001E00C2AAC28C2201
:104C1300AF5DEF3395E0FE7C0E7D10120E78EE3320
:104C230095E0FDFC906865E0F8A3E0F9A3E0FAA342
:104C3300E02FF52FEA3EF52EE93DF52DE83CF52C66
:104C4300754F01755018755180755201755306855E
:104C53002F54852E55852D56852C57E4F558F55937
:104C6300755C64C2DCD2AED20FC296D20D30210D78
:0D4C73007E217FC27C687D657B04123CDAE7
:014C80002211
:10369400300D03023816AC07754F487550618D51D3
:1036A400EB2480F55275530874442CF582E4346895
:1036B400F583E0600D74442CF582E43468F583E00E
:1036C40014F074442CF582E43468F583E0FF60124E
:1036D400EC25E024C1F582E43466F583E0A3E0FE42
:1036E40080027EFF8E54EF6012EC25E024C1F58247
:1036F400E43466F583E0FF7E0080047E007F7F8FE4
:10370400550C74442CF582E43468F583E0600D7440
:10371400442CF582E43468F583E014F074442CF509
:1037240082E43468F583E0FF6012EC25E024C1F5FF
:1037340082E43466F583E0A3E0FE80027EFF8E56C9
:10374400EF6012EC25E024C1F582E43466F583E0F1
:10375400FF7E0080047E007F7F8F570C74442CF51D
:1037640082E43468F583E0600D74442CF582E4341B
:1037740068F583E014F074442CF582E43468F5832E
:10378400E0FF6012EC25E024C1F582E43466F583A1
:10379400E0A3E0FE80027EFF8E58EF6012EC25E08D
:1037A40024C1F582E43466F583E0FF7E0080047E64
:1037B400007F7F8F590C74442CF582E43468F583C0
:1037C400E0600D74442CF582E43468F583E014F071
:1037D40074442CF582E43468F583E0FF6012EC2530
:1037E400E024C1F582E43466F583E0A3E0FE8002C0
:1037F4007EFF8E5AEF6012EC25E024C1F582E4349A
:1038040066F583E0FF7E0080047E007F7F8F5B127D
:023814004CEF77
:01381600228F
:104EB9008E2C8F2D9066D5E0FF2444F582E434686A
:104EC900F583E07002D322EF25E024C1F582E434B2
:104ED90066F583E0FEA3E0FF125266C006C007AF85
:104EE9002DAE2C125266C3D0E09FFFD0E09EFE1279
:104EF9005266AD697C00120EDFD3EF9403EE648035
:074F09009480400122D32235
:102D5D00E55E146077147003022DED147003022FDD
:102D6D00EF24036003022FF5A212B3921230122941
:102D7D007F031250E440103021487E217FD1E4FBC7
:102D8D00FDFC123CDA803B30210B7E217FF3E4FB0E
:102D9D00FDFC123CDA755E03227F051250E44010F3
:102DAD0030211F7E227F18E4FBFDFC123CDA8012DD
:102DBD0030210B7E227F37E4FBFDFC123CDA755E81
:102DCD000322755E019066D37403F0229066D3E002
:102DDD007003755E031252CA4003022FF5755E0231
:102DED00301211C2241250B3EF543F906877F0A304
:102DFD00E4F0800FC2241250B3EF540F906877F0B7
:102E0D00A3E4F0D2241250B3906878E02FF09068CC
:102E1D0077E03400F0201203022EEBE0FCA3E0FD7E
:102E2D00E4120BC47B0A7AD77923783C120A197BFA
:102E3D00667A66792078C212092890687912107C1A
:102E4D007530FF753122753259906879E0FCA3E039
:102E5D00FDA3E0FEA3E0F5368E358D348C337B017A
:102E6D007A68797D12294A30210D7E227F687C682F
:102E7D007D7D7B10123CDA906879E0F8A3E0F9A330
:102E8D00E0FAA3E0FBC000C001C002C003AC69E4DE
:102E9D00120BC9D003D002D001D000120A199068CC
:102EAD007912107C9066D5E0F52C7406F090687957
:102EBD00E0FCA3E0FDA3E0FEA3E0FF120BFD906696
:102ECD00CDEEF0A3EFF020AE0C124F59124428EFC7
:102EDD0060031200269066D5E52CF0022FEF906866
:102EED0077E0FCA3E0FDE4120BC47BBD7A527916AA
:102EFD00783D120A197BC57AFE790278C01209282D
:102F0D00C004C005C006C007906877E0FCA3E0FDD3
:102F1D00906877E0FEA3E0FF120E78AC06AD07E4F3
:102F2D00120BC47BF67A2479D67835120A19A804C7
:102F3D00A905AA06AB07D007D006D005D004120903
:102F4D002490687912107C7530FF753122753259D5
:102F5D00906879E0FCA3E0FDA3E0FEA3E0F5368EDA
:102F6D00358D348C337B017A68797D12294A302175
:102F7D000D7E227F907C687D7D7B10123CDA9068FF
:102F8D0079E0F8A3E0F9A3E0FAA3E0FBC000C001EB
:102F9D00C002C003AC69E4120BC9D003D002D0014A
:102FAD00D000120A1990687912107C9066D5E0F560
:102FBD002C7407F0906879E0FCA3E0FDA3E0FEA37C
:102FCD00E0FF120BFD9066CFEEF0A3EFF020AE0CFC
:102FDD00124F59124428EF60031200269066D5E572
:082FED002CF0756378E4F56730
:012FF50022B9
:1017E100201702C207301621C216E55C601BD55CCA
:1017F10018C206C20DC2AEC20F30210B7E227FB5C8
:10180100E4FBFDFC123CDAD29620140302199CC2BF
:10181100149066D3E0600214F090685DE0600214F9
:10182100F09066D9E07002A3E0600E9066DAE024E1
:10183100FFF09066D9E034FFF0E5636009D56306F7
:10184100756701E4F55E9066D2E0600214F090667F
:10185100ABE0600614F07002D20C9066D2E0600337
:1018610002199C30090BE567B40106122D5D0219BE
:101871009C30210B7E227FCFE4FBFDFC123CDA90F1
:1018810066D27405F09066AB7402F09066D5E024E0
:101891006BF582E43468F583E0701E9066D5E0FF55
:1018A100246BF582E43468F5837401F074AC2FF590
:1018B10082E43466F5837401F09066D5E004F0901B
:1018C10066D4E0FFA3E0C39F4002E4F09066D5E058
:1018D100FF24ACF582E43466F583E060611251D5F2
:1018E1009066D5E0FE24ACF582E43466F583EFF032
:1018F10074A32EF582E43466F583EFF02021030210
:10190100199C7E227FEB7C667DD57B01123CDA7FC0
:10191100321252A89066D5E024ACF582E43466F523
:1019210083E0600D7E237F06E4FBFDFC123CDA8040
:101931006A7E237F15E4FBFDFC123CDA805D906634
:10194100D5E0FF125230EF60249066D5E0FF24A36A
:10195100F582E43466F583E004F06402703D74AC12
:101961002FF582E43466F5837401F0802E9066D5FC
:10197100E0FF246BF582E43468F583E4F074A32F6F
:10198100F582E43466F583E4F0C20C30210D7E2348
:101991007F1D7C667DD57B01123CDAA297300A015E
:1019A100B3300B01B39290300F1A20AE17C20F3033
:1019B100210D7E237F3C7C007D5C7B01123CDAE4BF
:1019C100F55CD296300002C200201103021AE53004
:1019D100AE03021AE5C2119067DBE0600714F0E084
:1019E1007002D20830210D7E237F577C677DE0ABEA
:1019F10065123CDAE4FFFE752702E56524FEFDE58C
:101A010027C39D501474E02527F582E43467F583DC
:101A1100E02FFF2EFE052780E174DE2565F582E4C7
:101A21003467F583E06F6003021AE574DF2565F51D
:101A310082E43467F583E06E6003021AE57B01906E
:101A4100685E04F0A37468F0A37461F09066D6EB4D
:101A5100F0A37467F0A374DCF09067F5E09067DFA2
:101A6100F09067F4E09067DEF09067F3E0FE906736
:101A7100F2E07C002400FFEC3E9067DCF0A3EFF085
:101A81009067F8E0906861F09067F9E0640760039F
:101A9100C20A22D20A906861E004F09067F7E090F0
:101AA1006862F09067F6E0906863F0300836C2082B
:101AB1009066A2E09067DBF090685EE0FBA3E0FA3D
:101AC100A3E08B2F8A30F5319066D6E0FBA3E0FAD4
:101AD100A3E0F912458A90686512107CD224123D68
:101AE100E1124C13200403021B6B90685DE0707AD5
:0A1AF1009066D9E07002A3E0707067
:101AFB0090684CE0FCE4120BC9E4FBFA79C878421D
:101B0B00120A19E4FBFA79807842120B22120BFDB0
:101B1B009066D9EEF0A3EFF0E4F529906864E0F558
:101B2B002A9066D1E025E025E0F52B9066D4E0FF06
:101B3B00E529C39F501CAB2BAD2AAF291236947FDE
:101B4B00321252A874042529F5297404252BF52B80
:101B5B0080D930210B7E237F6DE4FBFDFC123CDA38
:101B6B009066D5E0FB246BF582E43468F583E06086
:101B7B0003021E3D200C03021E3DFD7F90125113EC
:101B8B005003021DEF7FAC125141E433F5289066F0
:101B9B00D5E0FB7D017F901251135003021DEF7FA7
:101BAB000A1252A8D2241250B38F27532780E5274D
:101BBB007003021DF29066D5E0FBE4FD7F9012519D
:101BCB00135003021DEF7FAA1251419066D5E0FB23
:101BDB007D017F901251135003021DEFE569D394E1
:101BEB00015003021C81C2241250B37E0090687511
:101BFB00EEF0A3EFF030E70BE02400F0906875E017
:101C0B0034FFF0906876E025E0F0906875E033F0F3
:101C1B00D2241250B3EF6007906876E04401F09045
:101C2B006875E0FEA3E0FFEE30E72FC3E49FFFE40F
:101C3B009EFE906875F0A3EFF0E569C313FD7C0081
:101C4B00120E78906875EEF0A3EFF0C3E49FFFE4FB
:101C5B009E906875F0A3EFF0803F906875E0FEA34F
:101C6B00E0FFE569C313FD7C00120E78906875EEFA
:101C7B00F0A3EFF08023C2241250B3906875E4F008
:101C8B00A3EFF0D2241250B3906876E030E70A2429
:101C9B0000F0906875E034FFF09066D5E0246BF5AA
:101CAB0082E43468F5837401F0C20C125298906888
:101CBB0075E0FEA3E0FF124EB9502C906875E0FE64
:101CCB00A3E0FF9066D5E0FD25E024C1F582E43466
:101CDB0066F583EEF0A3EFF074442DF582E43468DF
:101CEB00F583740AF08012202103021E3D7E237FB0
:101CFB008BE4FBFDFC123CDA22124F598F2820AEED
:101D0B000C124F59124428EF6003120026D21320F5
:101D1B002103021DF27E237FBF7C667DD57B0112E2
:101D2B003CDA7F321252A89066D5E025E024C1F54B
:101D3B0082E43466F583E0FEA3E0FF906869EEF081
:101D4B00A3EFF0EE30E74DE569D394014014EEF4C8
:101D5B00FEEFF42401FFE43EFEAD697C00120E8A17
:101D6B00801B9066D5E025E024C1F582E43466F54E
:101D7B0083E0F4FEA3E0F42401FFE43EFE906869E7
:101D8B00EEF0A3EFF07E237FD77C687D697B021298
:101D9B003CDA8053E569D39401401EE569FD7C0074
:101DAB009066D5E025E024C1F582E43466F583E046
:101DBB00FEA3E0FF120E8A80149066D5E025E02486
:101DCB00C1F582E43466F583E0FEA3E0FF90686919
:101DDB00EEF0A3EFF07E237FDF7C687D697B021240
:101DEB003CDA80031252989066D5E0FF24A3F5826B
:101DFB00E43466F583E004F074A32FF582E43466D3
:101E0B00F583E0D39402402A9066D5E0FF246BF56E
:101E1B0082E43468F5837401F074AC2FF582E434FA
:101E2B0066F5837401F074442FF582E43468F5830E
:021E3B00E4F0D1
:011E3D002282
:0352D1007F002239
:10507F000000001F003B005A0078009700B500D4D5
:10508F0000F301110130014E016D0000001F003CC3
:10509F00005B0079009800B600D500F401120131D1
:0450AF00014F016E3E
:064632008B328A3389344B
:10463800120F15AEF0244EF536EE34F8F53590002D
:1046480002120E3924FFF538E434FFF537E5362435
:1046580001FFE43535FE7C007D04120EDFAA06ABAF
:1046680007AE35AF367C017D6D120E78EF2BFDEE6F
:104678003AFCE53825E0FFE53733FE747F2FF582F5
:1046880074503EF5837401932DFFE4933CFEAB32E6
:10469800AA33900003120E397C002FFFEC3ECF2482
:1046A800FFCF34FFAB07FAAE35AF367D04120EDF0D
:1046B800ED64024C7012C3E5389402E537648094C7
:0C46C8008040050BBB00010AAE02AF03EE
:0146D40022C3
:10458A00124632EE3395E0FDFC7B807A5179017850
:10459A0000120F40C004C005C006C007AB2FAA30E6
:1045AA00A931900002120E39FFE4FCFDFE7B107A5D
:1045BA000EF9F8120F40D003D002D001D000EB2F31
:1045CA00FFEA3EFEE93DFDE83CFCC004C005C0062A
:1045DA00C007AB2FAA30A931900001120E39FFE4AF
:1045EA00FCFDFE7B3CFAF9F8120F40D003D002D052
:1045FA0001D000EF2BFFEE3AFEED39FDEC38FCA8B6
:10460A0004C005C006C007AB2FAA30A931120E207C
:10461A00FFE4FCFDFED003D002D001EB2FFFEE3AFF
:07462A00FEED39FDEC38FC48
:014631002266
:0A52A800E4FEEEC39F50030E80F8F1
:0152B20022D9
:10521300A2AF9224C2AF438E2075D2028F828E83B7
:0C522300E0FFE4F5D2538EDFA22492AF2E
:01522F00225C
:1051B100E5D220E0FBA2AF9224C2AF43D2028F829C
:1051C1008E83EDF075D25063D250A22492AFE5D216
:0351D10020E0FBE0
:0151D40022B8
:104B1B00E4FDED2401FFE433FE12521374372DF53F
:104B2B0082E43463F583EFF00DBD3FE6E4FDED2445
:104B3B007FFFE433FE125213742D2DF582E43461A2
:104B4B00F583EFF0742D2DF582E43461F583E0707D
:104B5B001B742D2DF582E43461F5837420F0742ED3
:104B6B002DF582E43461F583E4F080040DBD80BE45
:104B7B00E49061ACF0FDEDFF7E0012521374AD2D8D
:0D4B8B00F582E43461F583EFF00DBDFEE925
:014B980022FA
:104E08009080007480F090633763A201F583F58287
:104E180063A2017F081230D190633F63A2019080A2
:104E28008863A2017F0A1230D19080927407F0A3A0
:104E380074D0F0A37406F0906349E0FF9080B1F05D
:104E48009080E1EFF09080957455F0A3F090800089
:0A4E58007401F090800974F0F0225C
:104C8100908009E04410F09080A0E070609080A1D5
:104C91007482F09080A874FFF0A3F0A3F0A3F07FDA
:104CA100039080AEEFF0A374CBF09080007402F01B
:104CB10090689112108800000000906891E0908047
:104CC10040F0906892E0908041F0906893E090808D
:104CD10042F0906894E0908043F0A3E4F0A3F0A345
:0D4CE100F0A3F0908018F0A3F0A3F0A3F072
:014CEE0022A3
:104DAC00908009E04440F09080D17482F07F0390B1
:104DBC0080DEEFF0A374CCF09080027402F0906867
:104DCC009512108800000000906895E0908058F0D3
:104DDC00906896E0908059F0906897E090805AF037
:104DEC00906898E090805BF0A3E4F0A3F0A3F0A3AC
:0B4DFC00F0908030F0A3F0A3F0A3F0D3
:014E07002288
:104B9900908009E04420F09080B8E0706C9080B972
:104BA9007482F07F039080C6EFF07FCDA3EFF07F92
:104BB900039080C4EFF0A374CDF09080C074FFF02F
:104BC900A3F0A3F0A3F09080017402F09068991209
:104BD900108800000000906899E090804CF090687F
:104BE9009AE090804DF090689BE090804EF090683C
:104BF9009CE090804FF0A3E4F0A3F0A3F0A3F09021
:094C09008024F0A3F0A3F0A3F055
:014C1200227F
:104A97008C278D28A907EAFDE975F018A424ACFF37
:104AA700E5F034808F82F583EDF0EBFDE975F018C2
:104AB700A4FFAEF024ACFBEE34808B82F583A3ED2C
:104AC700F08528828C83E0FDEF24A8FFEE3480FE7A
:104AD7008F82F583EDF08528828C83A3E08F828E09
:104AE70083A3F0852882852783A3A3E0FDE975F0DA
:104AF70018A424A8FFE5F03480FE8F82F583A3A3D2
:104B0700EDF08528828C83A3A3A3E08F828E83A3F5
:044B1700A3A3F02242
:06487F008D2CAB07AA0618
:10488500908000E030E5079065797401F02290682A
:1048950091E0FCA3E0FDA3E0FEA3E0F5308E2F8DB3
:1048A5002E8C2DAE02AF038E838F8263A201E52F7E
:1048B500540744C0F58385308263A201AF2C1231C1
:1048C50043E4FCFDFEE530252CF530EE352FF52FC4
:1048D500ED352EF52EEC352DF52D908040E52DF09E
:1048E500A3E52EF0A3E52FF0A3E530F0908000744A
:1048F50020F0AF30AE2FAD2EAC2D90689112107C0C
:01490500228F
:064906008D27AB07AA0695
:10490C00908002E030E5079065797403F02290689E
:10491C0095E0FCA3E0FDA3E0FEA3E0F52B8E2A8D31
:10492C00298C28AE02AF038E838F8263A201E52A05
:10493C00540744D0F583852B8263A201AF27123133
:10494C0043E4FCFDFEE52B2527F52BEE352AF52A55
:10495C00ED3529F529EC3528F528908058E528F017
:10496C00A3E529F0A3E52AF0A3E52BF090800274CF
:10497C0020F0AF2BAE2AAD29AC2890689512107C94
:01498C002208
:0244DA008F272A
:1044DC00908001E030E5099065797402F07F00224C
:1044EC00906899E0FCA3E0FDA3E0FEA3E0F52B8E21
:1044FC002A8D298C2890667C63A201E52A540744F6
:10450C00C8F583852B8263A2017F06123159E52BF6
:10451C002406F52BE4352AF52AE43529F529E4356A
:10452C0028F52890657A63A201E52A540744C8F55A
:10453C0083852B8263A201AF27123159E4FCFDFE67
:10454C00E52B2527F52BEE352AF52AED3529F5290E
:10455C00EC3528F52890804CE528F0A3E529F0A34C
:10456C00E52AF0A3E52BF09080017420F0AF2BAE80
:0D457C002AAD29AC2890689912107CAF2759
:01458900220F
:103EE5009081E0E0F5270527052705270527052704
:103EF50005270527052705270527908010E0F52AC2
:103F0500A3E0F52BA3E0F52CA3E0F52D9081E1E0EE
:103F1500F52705270527052705270527052705274C
:103F2500052705270527908014E0F52EA3E0F52F3A
:103F3500A3E0F530A3E0F531E530B52C08E531B562
:103F45002D037F0022E4F527E530540744E0F5838F
:103F550085318263A20190637663A2017F081231E5
:103F65008990637863A2019062AE63A2017F061215
:103F750030D1906376E0F528A3E0F529E4F52790A4
:103F85006376E0702AA3E024F8F527E5305407446A
:103F9500E0F58385318274082582F582E43583F561
:103FA5008363A20190637663A201AF27123189AEC4
:103FB50028E4FCFDE5312529F531E5303EF530ED08
:103FC500352FF52FEC352EF52E908014E52EF0A328
:103FD500E52FF0A3E530F0A3E531F09080007440C3
:033FE500F0AF2713
:013FE80022B6
:10350D009081E6E0F52705270527052705270527DF
:10351D0005270527052705270527908028E0F52A8B
:10352D00A3E0F52BA3E0F52CA3E0F52D9081E7E0CA
:10353D00F52705270527052705270527052705272E
:10354D0005270527052790802CE0F52EA3E0F52F04
:10355D00A3E0F530A3E0F531E4F527E530B52C0A0D
:10356D00E531B52D05C21C023679E530540744F01E
:10357D00F58385318263A20190637663A2017F0892
:10358D00123189906376E0F528A3E0F529E5294508
:10359D002870099080027410F07F0022906683E0FD
:1035AD00FFF46030906378E06F6003023640906600
:1035BD0084E0FF906379E06F7079906685E0FF900D
:1035CD00637AE06F706D906686E0FF90637BE06FCD
:1035DD006031805F906378E0906683F0906379E06E
:1035ED00906684F090637AE0906685F090637BE05E
:1035FD00906686F090637CE0FFA3E090634ACFF085
:10360D00A3EFF0906376E0702AA3E024F8F527E5A8
:10361D0030540744F0F58385318274082582F58294
:10362D00E43583F58363A20190637663A201AF272E
:10363D00123189AE28E4FCFDE5312529F531E5305F
:10364D003EF530ED352FF52FEC352EF52EAF2DAE99
:10365D002CAD2BAC2AAB31AA30A92FA82ED312102A
:10366D006B40099080027410F07F002290802CE551
:10367D002EF0A3E52FF0A3E530F0A3E531F0908017
:06368D00027440F0AF27BB
:013693002214
:103817009081E3E0F52705270527052705270527D5
:103827000527052705270527052790801CE0F52A8A
:10383700A3E0F52BA3E0F52CA3E0F52D9081E4E0C0
:10384700F527052705270527052705270527052721
:10385700052705270527908020E0F52EA3E0F52F03
:10386700A3E0F530A3E0F531E4F527E530B52C0A00
:10387700E531B52D05C21D02396DE530540744E821
:10388700F58385318263A20190600463A2017F0EF4
:1038970012319F906004E0F528A3E0F52990600CB1
:1038A700E0FFF4604A90667CE0FEEF6E7079A3E07B
:1038B700FF90600DE06F706F90667EE0FF90600E86
:1038C700E06F706390667FE0FF90600FE06F705766
:1038D700906680E0FF906010E06F704B906681E02B
:1038E700FF906011E06F703FE4906013F0800890E4
:1038F700601374FFF0D2D9906004E0702AA3E0242B
:10390700F2F527E530540744E8F583853182740ED4
:103917002582F582E43583F58363A2019060046311
:10392700A201AF2712319FAE28E4FCFDE53125291E
:10393700F531E5303EF530ED352FF52FEC352EF529
:103947002EAF2DAE2CAD2BAC2AAB31AA30A92FA8A8
:103957002ED312106B5006E5294528700990800177
:103967007410F07F0022908020E52EF0A3E52FF061
:10397700A3E530F0A3E531F09080017440F0AF2764
:01398700221D
:043FE9008E2C8F2D5E
:103FED00908000E030E5079065797401F0229068CB
:103FFD0091E0FCA3E0FDA3E0FEA3E0F5338E328D4E
:10400D00318C30E533FFE5325407FEE42FF52FEE0A
:10401D0034C0F52E852F82F5837423F0052FE52FFF
:10402D007002052E532EC7F582852E83740AF00576
:10403D002FE52F7002052E532EC790633F63A2010B
:10404D00852E83852F8263A2017F0612314374066C
:10405D00252FF52FE4352EF52E852C83852D8263A6
:10406D00A201852E83852F8263A201123127E4FCE4
:10407D00FDFE906891E0F8A3E0F9A3E0FAA3E02F2C
:10408D00FFEE3AFEED39FDEC38FCEF2408FFE43E7F
:10409D00FEE43DFDE43CFC90689112107C9068912B
:1040AD00E0908040F0906892E0908041F0906893AD
:1040BD00E0908042F0906894E0908043F090800012
:0340CD007420F06C
:0140D00022CD
:0A3CDA008E308F318C328D338B3425
:103CE400908000E030E5079065797401F0229068D7
:103CF40091E0FCA3E0FDA3E0FEA3E0F53A8E398D4C
:103D0400388C37E53AFFE5395407FEE42FF536EEF3
:103D140034C0F535853682F5837423F00536E536EF
:103D2400700205355335C7F582853583740AF0056D
:103D340036E536700205355335C790633F63A201FB
:103D440085358385368263A2017F0612314374066A
:103D54002536F536E43535F535853083853182638E
:103D6400A20185358385368263A2011231278F3BF8
:103D7400EF2536F536E43535F535E534601785320B
:103D84008385338263A20185358385368263A201EC
:103D9400AF34123143E53B24082534F534FFE4FC09
:103DA400FDFEE53A2FF53AEE3539F539ED3538F5BE
:103DB40038EC3537F537908040E537F0A3E538F037
:103DC400A3E539F0A3E53AF09080007420F0AF3A0F
:0C3DD400AE39AD38AC3790689112107C0D
:013DE00022C0
:064298008E6A8F6B8D6C35
:10429E00908000E030E5079065797401F022906817
:1042AE0091E0FCA3E0FDA3E0FEA3E0F5728E718D1C
:1042BE00708C6FE572FFE5715407FEE42FF56EEE1C
:1042CE0034C0F56D856E82F5837423F0056EE56E50
:1042DE007002056D536DC7F582856D83EBF0056E2B
:1042EE00E56E7002056D536DC790633F63A2018545
:1042FE006D83856E8263A2017F061231437406259B
:10430E006EF56EE4356DF56D856A83856B8263A2FD
:10431E0001856D83856E8263A201AF6C1231437489
:10432E0008256CF56CFFE4FCFDFEE5722FF572EED0
:10433E003571F571ED3570F570EC356FF56F908068
:10434E0040E56FF0A3E570F0A3E571F0A3E572F020
:10435E009080007420F0AF72AE71AD70AC6F90684B
:04436E009112107C1C
:014372002228
:024A12008F49CA
:104A1400908000E030E5079065797401F022906899
:104A240091E0FCA3E0FDA3E0FEA3E0F54D8E4C8DE8
:104A34004B8C4AE54DFFE54C5407FEE42FFFEE3462
:104A4400C09062B563A201F5838F8263A201AF496E
:104A5400123143E4FCFDFEE54D2549F54DEE354CA0
:104A6400F54CED354BF54BEC354AF54A908040E575
:104A74004AF0A3E54BF0A3E54CF0A3E54DF090809C
:104A8400007420F0AF4DAE4CAD4BAC4A906891121F
:024A9400107C94
:014A960022FD
:0641B7008E278F28AB05E6
:1041BD00908000E030E5079065797401F0229068F9
:1041CD0091E0FCA3E0FDA3E0FEA3E0F52E8E2D8D86
:1041DD002C8C2BE52EFFE52D5407FEE42FF52AEE52
:1041ED0034C0F529852A82F5837423F0052AE52A42
:1041FD00700205295329C7F582852983EBF0052A1D
:10420D00E52A7002052990633F63A2018529838504
:10421D002A8263A2017F061231437406252AF52AEC
:10422D00E43529F5295329C7E527852A8285298370
:10423D00F0052AE52A700205295329C7F58285293B
:10424D0083E528F0052AE52A700205295329C7E5DB
:10425D002E240AF52EE4352DF52DE4352CF52CE420
:10426D00352BF52B908040E52BF0A3E52CF0A3E545
:10427D002DF0A3E52EF09080007420F0AF2EAE2D22
:0A428D00AD2CAC2B90689112107C50
:014297002204
:102FF600A907E7FFA805EF93C3966008403B74FC5A
:103006002FFF80F00F08EF93C3966008402B74FBE8
:103016002FFF80E00F08EF93C3966008401B74FAF9
:103026002FFF80D00F08EF93D3966008400B74F9FA
:103036002FFF80C01F1F1F1F1FEF54FEF80303F74B
:10304600E893FC08E893FD08E893FE08E893FF225E
:1030560009E993C39D6008402974FB29F980F109A9
:10306600E993C39E6008401A74FA29F980E209E9D7
:1030760093D39F6008400B74F929F980D319191965
:103086001919E9C313C313FF22740093F8ECC3980C
:103096004024701F740193F8EDC39840197014749E
:0E30A6000293F8EEC398400E7009740393F87D
:1030B400EFC39840037F00227F0122EDF8E6F00879
:1030C400A3DFFA22EDF8E0F608A3DFFA22E0A36317
:1030D400A201F0A363A201DFF475A2002263A2019E
:1030E400F0A363A20122E0A363A201F0A363A201FF
:1030F400E0A363A201F0A363A201E463A201F0A32D
:1031040063A201DFE175A20022E0A363A2016DFEC8
:10311400936CFDEE058393FC158363A201DFEA75CE
:10312400A200227F00E493A363A201F00F600CA32A
:10313400E583C2E3F58363A20180EA75A20022E07D
:10314400A363A201F0A3E583C2E3F58363A201DFD5
:10315400EE75A20022E0A363A201F0A3E583C2E41A
:10316400D2E3F58363A201DFEC75A20022E0A3633E
:10317400A201F0A3E58344F8C2E5F58363A201DF6D
:10318400EC75A20022E583C2E3F583E0A363A20108
:10319400F0A363A201DFEE75A20022E583C2E4D2AC
:0A31A400E3F583E0A363A201F0A3AA
:1031AE0063A201DFEC75A20022E58344F8F583E00B
:1031BE00A363A201F0A363A201DFEE75A20022F9C0
:1031CE0022C002C004C00612FFF0D006D004D00206
:0131DE0022CE
:0852B300D2947F141252A822CC
:0852BB00C2947F141252A822D4
:0F5288001252B3C225309202D2251252BBA22578
:0152970022F4
:025141008F2FAE
:10514300E4F530E52F30E704D2938002C293125284
:1051530088E52F25E0F52F0530E530C3940840E3BB
:05516300D293125288F6
:015168002224
:1050B300E4F52DF52E1252885002052DE52D25E03D
:1050C300F52D052EE52EC3940740EA1252885002AF
:1050D300052DC293302402D293125288D293AF2D5E
:0150E30022AA
:065113008F2C8D2D8B2E68
:105119001252BBD2937F141252A81252B3C2937F78
:10512900141252A81252BBE4FFE52E25E0FFE52C2C
:07513900252D2FFF1251414B
:01514000224C
:0250E4008F2D0E
:1050E6001252BBD2937F141252A81252B3C2937FAC
:1050F600141252A81252BB1252B3D2937F141252F8
:0C510600A81252BBE4FF252DFF125141FE
:01511200227A
:0752CA00309202C322D3223F
:105298001252BBC2937F141252A81252B3D2932255
:10092100020C69E86480F8E933E83360110460F08F
:10093100ED33EC337009E8FCE9FDEAFEEBFF22043C
:1009410060DED3EB9FEA9EE99DE8C2E78CF0C2F737
:1009510095F0400CE8CCF8E9CDF9EACEFAEBCFFB03
:10096100120C3485D0F05804700320D5B3E804701C
:10097100075002B2D5020C7392D5EC0460F7E4CCB7
:10098100C0E0C398F8603B94186008400DD0E0FBCC
:10099100020C4BE4FBFAC9FC8028E830E406E4C908
:1009A100FBE4CAFCE830E305E4C9CACBFCE8540720
:1009B1006010F8C3E913F9EA13FAEB13FBEC13FC2B
:1009C100D8F130F52FC3E49CFCEF9BFFEE9AFEEDCE
:1009D10099FDD0E0FBEF4E4D4C701222DB03020C6F
:1009E10070EC2CFCEF33FFEE33FEED33FDED30E721
:1009F100EB020C4BEF2BFFEE3AFEED39FDD0E0FBA5
:100A010050130BBB0003020C73ED13FDEE13FEEF4D
:080A110013FFEC13FC020C4B77
:100A1900EC4D6011E8497017ED33EC3304600DE4D7
:100A2900FCFFFEFD22E933E8330470F8020C691279
:100A39000C3458046009E4CC24815006285009027A
:100A49000C73284003020C70C0E0EB4A7044B98073
:100A590006D0E0FB020C5FEF4E701CBD8008EBFF77
:100A6900EAFEE9FD80EBE98DF0A4FEE5F0020B0258
:100A7900E9CDF9EAFEEBFFEF89F0A4FCE5F0CE89B8
:100A8900F0A42EFFE435F0CD89F0A42DFEE435F075
:100A99008067EF4E7005BD80D780C3EF8BF0A4ACA3
:100AA900F0EE8BF0A42CFCE435F0F8EF8AF0A42CDE
:100AB900E5F038FCE433CB8DF0A42CFCE5F03BF8F1
:100AC900EE8AF0A42CFCE5F038F8E433CF89F0A4E1
:100AD9002CFCE5F038CF3400CE89F0A42FFFE5F0E7
:100AE9003EFEE433C98DF0A42EFEE5F039CD8AF03F
:100AF900A42FFFE5F03EFEE43DFD33D0E0FB5007B7
:100B09000BBB000F020C73EC2CFCEF33FFEE33FE32
:060B1900ED33FD020C4B60
:100B1F00020C73EC5D046005E859047003020C6964
:100B2F00120C34580460F6EC4860F2EC7004FDFED1
:100B3F00FF22C860DB2481C85009C39860025006A9
:100B4F00020C709850CAF582E9294B4A7005AB82A6
:100B5F00020C5F75F0007C1A7880C3EF9BEE9AED64
:100B6F0099400DC3EF9BFFEE9AFEED99FDE842F021
:100B7F00DC23ACF0D0E0FFD0E0FED0E0FDAB822074
:100B8F00E7101BEB60BAEC2CFCEF33FFEE33FEEDFE
:100B9F0033FD020C4BE803F830E705C0F075F000A9
:100BAF00EF2FFFEE33FEED33FD40B830E7C280AAE2
:100BBF0075F020800E75F010800575F0087D007EB1
:100BCF00007F003392D530D50312105DEC33401007
:100BDF00EF33FFEE33FEED33FDEC33FCD5F0ED22BA
:0E0BEF00E5F0247EA2D513CC92E7CDCEFF22F6
:100BFD00EDD2E7CD33EC3392D524814006E4FFFEF0
:100C0D00FDFC22FCE4CFCECDCC24E0501174FF804E
:100C1D00EDC3CC13CCCD13CDCE13CECF13CF0470EB
:070C2D00F030D5DE02105D7E
:1028EE00E5442430F8E6054422782D302B0278306A
:1028FE00E475F0011210B9020E202024EB7F2ED2C7
:10290E00248018EF540F2490D43440D4FF30280B79
:10291E00EF24BFB41A0050032461FFE54560021591
:10292E00450548E54870020547302B0D782DE475B6
:10293E00F0011210B9EF020E66024F107403D22B83
:10294E008003E4C22BF5448B2D8A2E892FE4F545A6
:10295E00F547F548E54560077F2012292980F57572
:10296E0046FFC225C224C226C227C229C22AC22CB1
:10297E001228F7FF700D302B057F0012293AAF4851
:10298E00AE4722B4255FC2D5C2281228F7FF24D045
:10299E00B40A00501A75F00A784530D50508B6FF0E
:1029AE000106C6A426F620D5047002D22780D924AB
:1029BE00CFB41A00EF5004C2E5D228022C27D2253C
:1029CE0080C6D22480C0D22680BCD2D580BAD2296D
:1029DE0080B47F201229292026077401B5450040B6
:1029EE00F11228EEFF122929022962D22CD22A8056
:1029FE00951228EEFB1228EEFA1228EEF94A4B70C9
:102A0E0006791E7A2D7BFF20262EE545602A7E0054
:102A1E008E82758300120E3960060EEE654670F0DA
:102A2E00C2D5EBC0E0EAC0E0E9C0E0EE122C87D0E0
:102A3E00E0F9D0E0FAD0E0FB120E20FF60AAEBC066
:102A4E00E0EAC0E0E9C0E0122929D0E02401F9D083
:102A5E00E03400FAD0E0FBE5460460DCD546D980D0
:102A6E0087D22680A2122C6A60F7E5467001041206
:102A7E000C7EA946600DE546600914F546122D112F
:102A8E00EF60F3EA30E702F404C3995077EAF425D5
:102A9E00460430E701E404F546800D122C6A60C14D
:102AAE00EA05462546120C7EEA7843F630E701E445
:102ABE00254604D5460420290114122C87E4C0E0D3
:102ACE00122D117843E6601320E70714F612291130
:102ADE00802204F6D0E014C0E07F00122911E546F2
:102AEE0060071229081546800B302903122908D0D9
:102AFE00E0022962D0E00480C5122C6A60A0E5468F
:102B0E0004120C7E7843EAF6E546202902600104A1
:052B1E002404122C87C5
:102B230074FF04C0E0122D11122911E54620290279
:102B33006003122908D0E0B546E87F4512291B78C7
:102B430043E67F2B30E7047F2DF404C0E0122929EC
:102B5300D0E075F00A84C0F0122912D0E0122912D5
:102B6300022962791080027908C22AC22C8008D215
:102B7300D5790A8004790AC2D5E546047002F54680
:102B8300E4FAFDFEFF1228EEFC7B08202513122831
:102B9300EEFD7B1030240A1228EEFE1228EEFF7B96
:102BA30020EC3382D592D55013C3E43024069FFF23
:102BB300E49EFEE42025039DFDE49CFCE4CBF8C2E7
:102BC30025EC700CCFCECDCCE824F8F870F3801749
:102BD300C3EF33FFEE33FEED33FDEC33FCEB33FB9E
:102BE300994002FB0FD8E9EB302505F8D0E0C44843
:102BF300B225C0E00AEC4D4E4F78207B0070C2EA4C
:102C0300B5460040BCC0E0122C89D0F0D0E02025AE
:102C130004C4C0E0C4B225C0F0122912D0F0D5F02C
:102C2300EB0229621210C929FF532B665829D04C95
:102C330029CC422B6A4F2B72442B724929E5432B33
:102C430078552AA9462B07452A73472D3E5029D488
:102C53002D29D82E29FB2B29DC2329F9202D272ADE
:102C6300299448000029F3E546B4FF03754606128C
:102C730028EEFC1228EEFD1228EEFE1228EEFF7855
:102C83003C020CAD790AA2D5202714302909B910CA
:102C9300020404B9080104A2D5202A025001042029
:102CA30026689226B545005034C0E07F20302719AE
:102CB3007F30A226722A7229500F122CE0C226C23C
:102CC3002AC229C22C7F30800F302903E9C0E012C9
:102CD3002929302903D0E0F9D0E0B545CC302917B4
:102CE3007F30B9100C1229297F583028077F78804C
:102CF30003B908031229293026057F2D0229297FCC
:102D030020202CF87F2B202AF322922680CF7F00CD
:102D1300B407005005243CF8E6FF22286E756C6C5E
:102D23002900D2251228EE3025F8C225784530D562
:102D33000108F60229942D504349581228EE240322
:102D4300B405004001E4902D399312291A743A1204
:0A2D5300291AD227754504022B66E9
:100C3400E9D2E7C933E833F892D5EDD2E7CD33EC06
:070C440033FC5002B2D5227F
:100C4B00EC30E7100FBF000C0EBE00080DBD00040A
:100C5B000BEB6014A2D5EB13FCED92E7FD2274FFB6
:100C6B00FCFDFEFF22E480F8A2D574FF13FC7D800F
:030C7B00E480EF23
:100C7E00F920E72824F950037907E4F42402FB183D
:100C8E00DBFDE624FB5014E9600DE4F618E604F6ED
:0F0C9E00B40A08E4F6D9F57401F60A22C2D52289
:100CAD00ED33EC3392D5FA602AB4FF33EDC2E77B16
:100CBD00FF60067A0C79D2E4227A0C79DB20D50418
:100CCD007A0C79D6224E614E002B494E46002D49A5
:100CDD004E4600E47A08F608DAFC7B00740722E839
:100CED00C0E0ECC0E0EDC0E0EEC0E0EFC0E0EA75C2
:100CFD00F010A4CAABF075F04DA42BFBE435F0FC5D
:100D0D00EA2410FAEB34C5FBEC34D9FCEDC2E7FF55
:100D1D0075F056A4F42411C5F0F434C58FF0A42A4F
:100D2D00E5F03BE43CF620E714120DE0D0E0FFD0F7
:100D3D00E0FED0E0FDD0E0FC120B228014F4041292
:100D4D000DE0D0E0FFD0E0FED0E0FDD0E0FC120AD7
:100D5D0019D0E0F8E6FAEDD2E7CD33EC332482FB7F
:100D6D00E4C3CF33CFCE33CECD33CD33DBF37B07DF
:100D7D0075F00A846004F6081B0AE5F0F6088FF09A
:100D8D00740AA4FFACF08EF0740AA42CFEACF050E3
:100D9D00010C8DF0740AA42CFDE435F0F608DBDEB1
:030DAD00740722A6
:100DB0003F8000004120000042C80000447A00004B
:100DC000461C400047C35000497424004B189680CD
:100DD0004CBEBC205A0E1BCA6753C21C749DC5AEC4
:100DE000FB60065407601C2323120E0EEB54386080
:100DF00009120DFA120E09120A19ECF8EDF9EEFAC1
:100E0000EFCB22EB120E0980F1543803241C900D15
:100E1000B0FE93FC0EEE93FD0EEE930ECE93FF22EA
:030000000247F3C1
:0C47F300787FE4F6D8FD75817202483A28
:100E2000BB010689828A83E0225002E722BBFE02D0
:090E3000E32289828A83E4932203
:100E3900BB010CE58229F582E5833AF583E022506E
:100E490006E92582F8E622BBFE06E92582F8E222B8
:0D0E5900E58229F582E5833AF583E49322D2
:100E6600BB010689828A83F0225002F722BBFE016B
:020E7600F32265
:100E7800EF8DF0A4A8F0CF8CF0A428CE8DF0A42E8E
:020E8800FE2248
:100E8A00BC000BBE0029EF8DF084FFADF022E4CC4C
:100E9A00F875F008EF2FFFEE33FEEC33FCEE9DEC15
:100EAA00984005FCEE9DFE0FD5F0E9E4CEFD22ED5B
:100EBA00F8F5F0EE8420D21CFEADF075F008EF2FA5
:100ECA00FFED33FD4007985006D5F0F222C398FD96
:050EDA000FD5F0EA2233
:100EDF00C2D5EC30E709B2D5E4C39DFDE49CFCEE2E
:100EEF0030E715B2D5E4C39FFFE49EFE120E8AC30E
:100EFF00E49DFDE49CFC8003120E8A30D507C3E409
:060F0F009FFFE49EFE229C
:100F1500BB010A89828A83E0F5F0A3E022500687A7
:100F2500F009E71922BBFE07E3F5F009E319228969
:0B0F3500828A83E493F5F0740193229C
:100F4000E88FF0A4CC8BF0A42CFCE98EF0A42CFC50
:100F50008AF0EDA42CFCEA8EF0A4CDA8F08BF0A4CE
:100F60002DCC3825F0FDE98FF0A42CCD35F0FCEB2D
:100F70008EF0A4FEA9F0EB8FF0A4CFC5F02ECD39F2
:0F0F8000FEE43CFCEAA42DCE35F0FDE43CFC225F
:100F8F0075F008758200EF2FFFEE33FECD33CDCC19
:100F9F0033CCC58233C5829BED9AEC99E58298409C
:100FAF000CF582EE9BFEED9AFDEC99FC0FD5F0D679
:100FBF00E4CEFBE4CDFAE4CCF9A88222B800C1B9A3
:100FCF000059BA002DEC8BF084CFCECDFCE5F0CBE1
:100FDF00F97818EF2FFFEE33FEED33FDEC33FCEB1A
:100FEF0033FB10D703994004EB99FB0FD8E5E4F9D5
:100FFF00FA227818EF2FFFEE33FEED33FDEC33FCC2
:10100F00C933C910D7059BE99A4007EC9BFCE99AB5
:10101F00F90FD8E0E4C9FAE4CCFB2275F010EF2FFA
:10102F00FFEE33FEED33FDCC33CCC833C810D707FA
:10103F009BEC9AE899400AED9BFDEC9AFCE899F835
:0E104F000FD5F0DAE4CDFBE4CCFAE4C8F922C8
:0E105D00C3E49FFFE49EFEE49DFDE49CFC22A4
:10106B00EB9FF5F0EA9E42F0E99D42F0E89C45F0DB
:01107B002252
:0C107C00ECF0A3EDF0A3EEF0A3EFF022E7
:10108800A8828583F0D083D08212109F12109F12FD
:10109800109F12109FE473E493A3C583C5F0C58322
:1010A800C8C582C8F0A3C583C5F0C583C8C582C8B2
:0110B8002215
:1010B900FAE6FB0808E6F925F0F618E6CA3AF62238
:1010C900D083D082F8E4937012740193700DA3A3B6
:1010D90093F8740193F5828883E4737402936860CA
:0610E900EFA3A3A380DFCA
:10526600C3EE6480948040028007C3E49FFFE49EFF
:02527600FE2216
:1031DF008B288A29892AE4F534F533F532F531F550
:1031EF002FF530E52C452D452B6012EBC0E0EAC0E2
:1031FF00E0E9C0E0AB2BAA2CA92D1210EFAB2805EC
:10320F002AE52AAA297002052914F9120E20F5358C
:10321F00C394094007E535D3940D40E1E5356420AB
:10322F0060DBE535B42D054330038016E535B42B4F
:10323F0005433001800C74FF252AF52A74FF3529C8
:10324F00F529E52E60046410703FAB28AA29A92A3E
:10325F00120E2064306009E52E702E752E0A80291B
:10326F00900001120E39FF64786004EFB4581343D5
:10327F003001752E107402252AF52AE43529F52917
:10328F008007E52E7003752E08AB28052AE52AAABC
:10329F00297002052914F9120E20F535C3946140E7
:1032AF000AE535D3947A50035335DF74D02535F5BD
:1032BF0035C3940A400CE5359411406D74F92535EA
:1032CF00F535E535D3952E5060433001853439857A
:1032DF003338853237853136AF2E7E00E4FCFDABB7
:1032EF0034AA33A932A831120F40C8ECC8C9EDC9AE
:1032FF00CAEECACBEFCBE4FCFDFEEB2535F534EE81
:10330F003AF533ED39F532EC38F531AF34AE33AD44
:10331F0032FCAB39AA38A937A836D312106B500339
:10332F00023298433004023298E53020E003E48003
:10333F002DE52C452D452B601EAB28E52A24FFF9E2
:10334F00E52934FFFAEBC0E0EAC0E0E9C0E0AB2BBF
:10335F00AA2CA92D1210EFE53030E20774FFFFFE03
:10336F00FDFC22E530AF34AE33AD32AC3130E1038A
:04337F0002105D22B9
:1047FF00021159E493A3F8E493A34003F68001F266
:10480F0008DFF48029E493A3F85407240CC8C333BA
:10481F00C4540F4420C8834004F456800146F6DF89
:10482F00E4800B0102040810204080904F9EE47E2C
:10483F00019360BCA3FF543F30E509541FFEE4937E
:10484F00A360010ECF54C025E060A840B8E493A345
:10485F00FAE493A3F8E493A3C8C582C8CAC583CA70
:10486F00F0A3C8C582C8CAC583CADFE9DEE780BE28
:014FDD0000D3
:1010EF00BB011A89828A83D0F0D0E0F8D0E0F9D022
:1010FF00E0FAD0E0FBE8C0E0C0F00211475016E97B
:10110F00F8D083D082D0E0F9D0E0FAD0E0FBC082F3
:10111F00C08302113EBBFE16E9F8D083D082D0E027
:0F112F00F9D0E0FAD0E0FBC082C0830211502259
:09113E00EBF608EAF608E9F622D6
:09114700EBF0A3EAF0A3E9F022A9
:09115000EBF208EAF208E9F222D0
:00000001FF
